:080000000C946A000C9400004E
:100008000C9400000C9400000C9400000C94000068
:100018000C9400000C9400000C9400000C94000058
:100028000C9400000C9400000C9400000C94000048
:100038000C9400000C9400000C94CC000C9400006C
:100048000C9499000C9400000C9400000C9400008F
:100058000C9400000C9400000C9400000C94000018
:100068001027E80364000A000100001000011000D6
:100078000100000000000A0000000000000000006D
:100088000000000000000000000000000000000068
:100098000000000000000000000000000000000058
:1000A800000000000000000A0A0A0A0A0A0A0A0AEE
:1000B8000A0A0A0A0A0A0A00020002007A00020072
:1000C80004007C00010009037E000000F894EE277C
:1000D800EFBBF1E0F5BFE5BF8DE0A2E0BB27ED93F4
:1000E8008A95E9F780E098E0A0E0B1E0ED93019708
:1000F800E9F7E0ECF0E085919591009761F0A59122
:10010800B59105901590BF01F00105900D920197EA
:10011800E1F7FB01F0CFE8E0EEBBEFEFEDBFE8E081
:10012800EEBFC0E0D3E00C947A03AA93EA93FA9363
:10013800EFB7EA931A930A931091C0000091C60092
:10014800E12FEC71E9F4E091E803EF5FE093E80355
:10015800E150F0E0E153FC4F0083A091E803A9319E
:1001680019F4E0E0E093E803A091EA03AF5FA093FD
:10017800EA03A93129F4E0E0E093EA03689435F84A
:1001880009911991E991EFBFF991E991A991189510
:100198000A921A926A937A938A939A93AA93BA9331
:1001A800EA93FA93EFB7EA93E0913903F0913A03AF
:1001B8003196E0933903F0933A030E94B41EE1E5C7
:1001C800F1E00E940E280E2E0E94B41EE3EAF2E02F
:1001D8000E940E28E02909F4EFC1A0913703B091DD
:1001E8003803E4E1F0E00E9420280E2EE091060397
:1001F800F0E074970E9414280E22A0911E03EEE0EE
:100208000E940428E02121F0E0911E03EF5F03C063
:1002180025FC03C0E0E0E0931E03A0911E03AE306E
:1002280011F4689425F8E0913703E0930603A09150
:100238002703A13029F4F79B02C0F79801C0F79A69
:10024800E1E02E260E94B91E0E94C21EE093B3036D
:10025800F093B4036093B5037093B6030E94C91E6C
:10026800A7E9B3E00E94CE1E0E94D51EA3ECB3E01E
:100278000E94CE1E0E94DA1E0E94E31E0E943A27A8
:10028800E0939703F09398036093990370939A030C
:10029800A091C303B091C4038091C5039091C60394
:1002A800E0E0F0E060E772E40E943A27E093C303DD
:1002B800F093C4036093C5037093C6030E94E81EBD
:1002C8000E94ED1E0E2E0E94F21E0E94ED1EE021DD
:1002D80061F1E091C303F091C4036091C50370918B
:1002E800C6030E94DA1E0E943A27E093BF03F093E8
:1002F800C0036093C1037093C2030E94F71EABE46E
:10030800B3E00E94001FA091BF03B091C003809189
:10031800C1039091C2030E94C21EE0939F03F09311
:10032800A0036093A1037093A2030E94051F0E947B
:10033800161F0E949C26E093A703F093A8036093DE
:10034800A9037093AA030E94051F0E941F1F0E9401
:100358009C26E093CB03F093CC036093CD0370937A
:10036800CE030E94281F0E94311F0E94441FA3E849
:10037800B3E00E942B260E9402290E94281FAAE0AF
:10038800B0E080E090E00E9446280E941F1F0E9473
:1003980060260E947F2770F0E0E0E093CB03E093B3
:1003A800CC03E093CD03E093CE030E94491F31961E
:1003B8000E944E1F0E94531FA091AB03B091AC0343
:1003C8008091AD039091AE030E9462260E94EC26B4
:1003D800DF01CB010E94C21EE093B703F093B8037C
:1003E8006093B9037093BA030E945C1F0E949C2615
:1003F8000E94651F0E94281FA5E2B0E080E090E0FF
:100408000E946E1FABE6B3E00E947D1F0E94B91EDA
:100418000E9458293CF5A091B703B091B803809188
:10042800B9039091BA030E94821F7F936F93FF9341
:10043800EF93A091B303B091B4038091B503909169
:10044800B6030E94821FAF91BF918F919F910E9426
:100458003A27E093AF03F093B0036093B10370932E
:10046800B20309C0E0E0E093AF03E093B003E09388
:10047800B103E093B2030E94891FACE2B3E00E948B
:100488002926EC930E94921F0E949B1F0E949C2683
:100498000E94A41FE0919703F0919803609199033B
:1004A80070919A030E94AD1F0E947F2768F5E09122
:1004B8009F03F091A0036091A1037091A2030E9491
:1004C800AD1F0E949C26E0939B03F0939C036093CE
:1004D8009D0370939E030E94AD1F0E94B61F0E9449
:1004E8009526DF01CB010E94F71E0E943A27A0E063
:1004F800B0E081E695E40E94EC26A7E6B3E00E940E
:100508007D1F689424F802C0E0E12E260E94921F05
:100518000E94BF1F0E949C26E093A303F093A403AC
:100528006093A5037093A6030E94BF1FE0E0F0E06C
:1005380060E87FE30E947F2709F008F412C0E09387
:10054800A303E093A403E093A503E093A6030E940A
:10055800C81FEF5FFF4F6F4F7F4F0E94D11F0E9450
:10056800DA1F0E94E01FA034E2E4BE07EFE08E0726
:10057800E0E09E0778F0E0E0E0935903E0935A0347
:10058800E0935B03E0935C03AAE3B0E00E94E91FF9
:100598000E942D290E949B1F0E94EE1FABE3B3E02F
:1005A8000E94001FA0911C03AC3308F4F298A0919C
:1005B8001C03AC3309F4F29A0E94B41EA33AE2E099
:1005C800BE0709F06AC0A0911B030E94F21F0E9497
:1005D800F71F0E94E91F0E9426280E940020E021A0
:1005E80091F0E0911C03EF5FE0931C03E0911B0383
:1005F800F0E03296A0911C03B0E0EA17FB0719F46B
:10060800ECE3E0931C03E0E0E0933903E0933A0362
:10061800C3940E940720E8E5F2E00E941A280E2EF3
:100628000E940C20E021E9F0E0914F03F091500383
:100638003196E0934F03F09350030E9407200E94E5
:100648001120EA1BFB0BE0935503F09356030E941D
:10065800F71F0E9458292CF4E0E0E0934F03E09341
:100668005003ECE3EC15C9F4CC24E0910003EF5FF0
:10067800E0930003A0910003AC3379F4E0E0E09349
:100688000003E0910103EF5FE0930103A0910103F0
:10069800A43119F4E0E0E0930103E991EFBFF99187
:1006A800E991B991A9919991899179916991199053
:1006B80009901895AA93E881E066E0937C0085E2AA
:1006C8008A95F1F7E0917A00E064E0937A00E0918E
:1006D8007A00E071E1F3E0917A00E061E0937A005A
:1006E800E0917800F091790021960895EF9722978C
:1006F8008FE3A2E0B0E0E0E8F0E00E946D29FF247B
:1007080001E021E0E0E8E0936100E0E0E0936100CF
:10071800EFE0E4B9E1E0E5B9E0E0E7B9E4E0E8B941
:10072800EAEFEAB9E7EEEBB9E0E0E4BDE3E0E5BD06
:10073800E0E0E6BDE7BDE8BDE1EAE0938000E2E085
:10074800E0938100E0E0E0938500E0938400E0938B
:100758008700E0938600E0938900E0938800E093A7
:100768008B00E0938A00E093B600E1EAE093B000E2
:10077800E2E0E093B100E0E0E093B200E093B30080
:10078800E093B400E1E0E0936E00E0E0E0936F00F6
:10079800E0937000E0936900EDBBE0936800E0939C
:1007A800C000E8E9E093C100E6E0E093C200E0E0C1
:1007B800E093C500E7E4E093C400E0E8E0BFE0E0D0
:1007C800E0937F00E0937E00E0E6E0937C00E7E2C0
:1007D800E0937A00E0E0E0937B00ECBDE093BC009E
:1007E8007894A4E1B0E00E94F2255F9A0E94162056
:1007F8000E9426200E943320EAE09E1620F4A8E2F8
:10080800B0E00E943D20EAE08E1650F4AEE2B0E07F
:100818000E943D20A6E3B0E00E943D20689426F89F
:10082800EAE0AE1618F4689430F827F8689433F8BC
:10083800E3E1E09310030E9442200E9449200E94B5
:100848005020E8ECF0E0E0936103F0936203A0E04D
:10085800B0E00E942129E0931103A1E0B0E00E94DA
:100868002129E0931203A2E0B0E00E942129E0933D
:100878001303A3E0B0E00E942129E0931503A4E04C
:10088800B0E00E942129EF8BA5E0B0E00E94212969
:10089800E88FA6E0B0E00E942129E98FA7E0B0E048
:1008A8000E942129E0931603A8E0B0E00E942129C4
:1008B800E0931703A9E0B0E00E942129E093180310
:1008C800F798F198AAE0B0E00E942129E0931B0371
:1008D800A6E2B0E00E941D290E945720A4E1B0E0E2
:1008E8000E942129EB8BA5E1B0E00E942129EC8B25
:1008F800A6E1B0E00E942129ED8BABE0B0E00E94B8
:100908002129EF87ACE0B0E00E942129E88BADE017
:10091800B0E00E942129E98BAAE2B0E00E941D29DB
:10092800ED83FE83AEE0B0E00E942129E093280326
:10093800AFE0B0E00E942129E0932A03A0E1B0E0F3
:100948000E942129E0932903AAE3B0E00E94192913
:100958000E94D11FA8E2B0E00E941D29A3E9B3E0DC
:100968000E945C200E94B61FABE3B3E00E94001F08
:100978000E949B1F0E94E31E0E943A270E94A41F08
:10098800A1E1B0E00E9421293E2FACE2B0E00E9434
:100998001D29E987FA87A2E1B0E00E942129EB8F9F
:1009A800A3E1B0E00E942129EA8FAEE2B0E00E9404
:1009B8001D29A7EAB3E00E945C20A6E3B0E00E94EC
:1009C8001D29A7ECB3E00E945C200E945C1F0E94D6
:1009D800E31E0E943A270E94651FA0E3B0E00E9430
:1009E8001D290E946320A4E3B0E00E941D290E94F3
:1009F800E1270E946820A7E1B0E00E9421290E9417
:100A0800682923F8A2E3B0E00E941D290E94712002
:100A1800A8E1B0E00E942129E0930803A9E1B0E031
:100A28000E942129E0930A03AAE1B0E00E9421294B
:100A3800E0930B03ABE1B0E00E942129E0930C03A3
:100A4800ACE1B0E00E942129E0930D03ADE1B0E0F4
:100A58000E942129E0930E03AEE1B0E00E94212913
:100A6800E0931F03AFE1B0E00E942129E093200347
:100A7800A0E2B0E00E942129E0932103A1E2B0E0C6
:100A88000E942129E0932203A2E2B0E00E942129DA
:100A9800E0932303A3E2B0E00E942129E09324031A
:100AA800A4E2B0E00E942129E0932503A5E2B0E08A
:100AB8000E942129E0932603A8E3B0E00E941D29A3
:100AC8000E944E1FA0910303A43128F4E091030370
:100AD800EF5FE0930303A0910303A431A1F4E0E0E6
:100AE800E0932E03E0932F03EBE0F0E0E093530351
:100AF800F0935403E8EBE0933003E0E0E093E8037D
:100B0800EAE0E0930303A091E803AB30C1F4E0917D
:100B1800D203E0932E03E091D303E0932F03E091F7
:100B2800D403F0E0E0935303F0935403E091D5032A
:100B3800E0933003E0E0E093E803E0930303A0913F
:100B4800E803AC30C0F0E0E0E093CF03E093D003DB
:100B5800E093D103E093D203E093D3030E944220B1
:100B6800E0E0E093D603E093D703E093D803E09363
:100B7800D903E093E803E8EC5E1630F45394E4E11B
:100B8800E51511F4E1E04E2EA4E1B0E00E94F22553
:100B98000E9476203B9798F1A0E00E947F2066276C
:100BA80077270E9486200E94531FA8EEB3E080E0BA
:100BB80090E00E947128DF01CB010E948F206627F8
:100BC80077270E94B3280E948620E0910903EF5FEF
:100BD800E0930903E0910803A0910903AE1768F0B8
:100BE8000E94531FE0937F03F09380036093810377
:100BF80070938203E0E0E0930903E894F3F8E7E2F6
:100C0800E0937A000E941620A2E00E947F20DF0174
:100C1800E5E0F0E00E947628BE2E0E9494200E9413
:100C280026200E949B200E949420A5E00E94A520D7
:100C38001E2FE7E2E0937A000E947620DE2E0E94C3
:100C480094200E943320E7EAE0937A00A6E00E940D
:100C5800A520ED87E7E2E0937A00E1E0E51591F55C
:100C68000E94AA20E2E3F0E00E9420280E2E0E94B3
:100C7800AF200E941A28E02111F0E5E0EC87A12FAF
:100C8800E2E30E9409280E2EEAEF0E940428E021E0
:100C980011F0E6E0EC870E94AF200E9420280E2E7B
:100CA8000E94B320E02911F0E7E0EC87A12FEAEFDA
:100CB8000E9409280E2EEEE10E940428E02911F076
:100CC800E8E0EC870E94AF200E9420280E94B9200B
:100CD80039F0E1E0EC87E8E2F0E00E94C52007C0C7
:100CE8000E94B3200E94B92011F0E2E0EC87A12F06
:100CF800EAEF0E9409280E94B92011F0E3E008C039
:100D0800A12FEEE10E9404280E94B92019F0E4E026
:100D1800EC871CE3AC850E94CA20AC85E7E00E9402
:100D2800EB270E2AE1E00E94EB270E2AE2E00E9460
:100D3800EB27E02929F0E12FF0E00E94C52018E216
:100D4800AC850E94CF20AC85E8E00E94EB27E02923
:100D580009F018E20E94D4200E94DA200E94042898
:100D6800E021D1F06894F3F8013021F4F398F49A73
:100D780002E012C0023059F4F498F59AA98DA13016
:100D880010F003E003C0F598F39A01E005C00330C2
:100D980019F4F598F39A01E00E94AA20D39708F471
:100DA80057C00E94E4200E94E920E02F0E94F02012
:100DB80020F0E8ECF0E00E94C520E02F0E9400211E
:100DC8000E941021AC91A13008F441C00E94172163
:100DD8000E9420210E9463294CF40E9410210E9445
:100DE8002C210E94AB270E94372123C00E9440215A
:100DF8000E944221EF930E9440210E944B21AF9113
:100E0800EA2379F00E9410210E942C210E94B02729
:100E1800A0936F03B0937003809371039093720350
:100E280008C00E9440210E9454211CF00E945E21AB
:100E38000EC0A0916F03B0917003809171039091DF
:100E480072030E946D210E94B3280E94C52004C02D
:100E58000E9472210E945E210E9478210E947E21B8
:100E68000E220E948321E02139F0E0913503E093BE
:100E78001D036894F0F821F80E94E420309721F4CB
:100E8800E0E0E0931E0306C0A0911E03A23010F418
:100E9800E89425F80E94E420E0933703F0933803A0
:100EA8000E94E420309719F4E89421F815C0A0E0D6
:100EB80021FCA1E0E0E00E94EB270E2EA0911D038B
:100EC800E0E00E940928E02139F0E0E0E0931D030A
:100ED8000E947221E89422F8E09105030E94AA205A
:100EE800F0E0AE17BF0720F0E0913503E09305036B
:100EF800E0910503F0E035970E94AA20AE17BF07DE
:100F0800B0F4E0913503E0930503A0E025FCA1E0EF
:100F1800E1E00E94EB270E2E0E948A2141F0E2E0D8
:100F2800E0932B03E89425F8E0E0E0931E03A091FA
:100F38001D03A13080F0689422F80E94E420A0915B
:100F48001D03B0E0AE17BF0728F0E0911D03F0E0E5
:100F58000E94C52002C0E89422F80E9492210E94B3
:100F680095210E9436280E22A09128030E949C21D8
:100F78001E2E0E9492210E9495210E942E280E2248
:100F8800A09129030E949C211E2A0E949221A12F30
:100F9800E2E30E940928E021E12979F00E94722108
:100FA800A0912B03A13021F4EAE0F0E00E94C520D3
:100FB800E0912B03E150E0932B030E94A1210E2224
:100FC800A0E031FCA1E00E949C2131F0689431F846
:100FD8000E94E4200E94B7210E94A121E02161F132
:100FE8000E94BC210E94C421A4F0A0917B03B0916F
:100FF8007C03ED81FE81EA1BFB0BA3E0B0E00E94BD
:101008006C280E94CC21AE1BBF0BA0936303B09346
:1010180064030E94BC210E9458292CF40E94D1210B
:1010280032970E94B721A0916403AA232AF4E0E032
:10103800E0936303E09364030E94D6210E945E2933
:1010480074F50E94D6210E94B0270E94C42174F032
:10105800AD81BE81E0917B03F0917C03EA1BFB0B21
:101068000E94CC21EA0FFB1F0E94B7210E94D621C3
:101078000E94B027A230E0E0BE07E0E08E07E0E083
:101088009E072CF00E94D12131960E94B7210E9420
:10109800CC21A93CE0E0BE0714F00E9449200E9440
:1010A800D1210E94AA20AE17BF0710F4E89431F8A6
:1010B8000E94D1210E94AA20EA17FB0720F40E946F
:1010C800D1210E94C5200E94E3210E94A5270E2E4F
:1010D800A0E032FCA1E00E949C2141F0689432F823
:1010E8000E94F221E0936503F09366030E94E321D6
:1010F8000E947F2709F008F435C00E94F721DF011C
:10110800CB01E0E0F0E060E070E40E947F2709F0A6
:1011180008F410C00E94F721DF01CB01E985FA85A8
:101128000E9406220E940D220E941222A5E6B3E028
:101138000E947D1F0E94F7210E944E2954F4EB8DD6
:10114800F0E00E940D22AE1BBF0BA0936503B09385
:101158006603A0916603AA232AF4E0E0E0936503FE
:10116800E09366030E94E3210E947F27D0F50E9446
:101178001722DF01CB01E0E0F0E060E470E40E94B8
:101188007F2709F008F416C00E941722A0E0B0E0FB
:1011980080EA90E40E94EC26DF01CB010E94222223
:1011A8000E94E1270E9462260E949C26A5E6B3E0E1
:1011B8000E947D1F0E9417220E944E2954F4EA8D36
:1011C800F0E00E940D22EA0FFB1FE0936503F09305
:1011D80066030E940D22A13DE7E0BE0714F00E94BD
:1011E80050200E94F221DF010E942222AE17BF0781
:1011F80010F4E89432F80E94F221DF010E942222C2
:10120800EA17FB0720F40E940D220E9427220E9461
:101218002C220E9436280E2EA0E034FCA1E00E9469
:101228009C2131F0689434F80E94F2210E94332204
:101238000E942C220E945E295CF50E9438220E949E
:10124800C4219CF0E0911203F0E0A0917703B091E3
:101258007803AE1BBF0BE3E0F0E00E944122AE1B17
:10126800BF0BA0936D03B0936E030E9438220E94B7
:1012780058292CF40E94482232970E943322A091C8
:101288006E03AA232AF4E0E0E0936D03E0936E0373
:101298000E942C220E9463298CF50E944D22A430C2
:1012A800E0E0BE07E0E08E07E0E09E078CF0A0914A
:1012B8001203BB27E0917703F0917803AE1BBF0BB5
:1012C800E2E0F0E00E944122EA0FFB1F0E94332275
:1012D8000E944D220E9458292CF40E9448223296DE
:1012E8000E943322A0916D03B0916E03A13DE7E007
:1012F800BE0724F0E0EDF7E00E9433220E94F221BD
:10130800DF010E944822AE17BF0710F4E89434F8B2
:101318000E94F221DF010E944822EA17FB0730F4FD
:10132800A0916D03B0916E030E9427221333D8F069
:10133800A0911D03A13018F0E2E0E0932B03E0E058
:10134800E0931D03E12FF0E0F2970E94E1270E944D
:101358006226A6EFB8E28CE99FE30E94EC260E9481
:1013680029261E2F01C010E00E94E420EB83FC8395
:10137800AB2DE4E60E9404280E2EA0E0F099A1E02F
:10138800E1E00E94EB270E9400200E22AA81EDE5F1
:101398000E94F027E0211E2E0E9411200E940720A3
:1013A8000E940E280E945D220E940C20E021E12963
:1013B80009F1E0913B03F0913C03A8E2B0E00E9400
:1013C80065220E946B220E945C1F0E94EE1F0E94F1
:1013D80078220E94491FA8E3B0E00E943529A4E6BC
:1013E800B0E00E94F2255F98A8EEB3E00E94F225D3
:1013F8005F98FECFAA2D0E947D220E947E21E021C7
:1014080031F0E894F2F827F8E0E0E09334030E9422
:1014180082220E947E21E02171F0E0913403EF5F87
:10142800E0933403A0913403AA3029F4E0E0E09378
:101438003403E09327030E9482220E948F220E9495
:101448007E21E02171F06894F2F8E0912703EF5FC4
:10145800E0932703A0912703A33019F4E1E0E09378
:101468002703E0912703E03029F4E0E0E093B4009B
:10147800F7980FC0A0912703A13019F4E091180341
:1014880006C0A0912703A23021F4F79AEFEFE0936A
:10149800B4000E94AA200E94ED1E0E2EA12FE0E0AB
:1014A8000E9409280E220E948A2101F1E09104037A
:1014B800EF5FE0930403A0910403E5E00E9409288C
:1014C8000E2EE4E10E940428E02141F0E09104039B
:1014D800E170AFEFEA02F001E093B400A0910403D9
:1014E800A03118F0E0E0E093040326C0A0E030FC4F
:1014F800A1E0E1E00E94EB270E2EA09127030E94B5
:101508009C21D1F0E0913303EF5FE0933303A09186
:101518003303A13019F4EFEFE093B400A091330343
:10152800A33019F4E0E0E093B400A0913303A430B1
:1015380019F4E0E0E0933303E0911703E093B3007C
:10154800EAE0E81518F4E894F1F826F80E949722E2
:10155800A0E026FCA1E00E949D22A0E0F1FCA1E011
:101568000E949D220E947E21E02139F16894F1F8C1
:10157800E0910F03EF5FE0930F03E0E0EB87AB85AB
:10158800A53088F40E94A222A081A13018F0E5E0DD
:10159800EB8705C0E0910F03EF5FE0930F03EB8546
:1015A800EF5FEB87ECCFA0910F03A53018F0E0E0D8
:1015B800E0930F030E94A22220810E949722A0910B
:1015C8001A03EFEF0E940428E02121F0E0911A03AA
:1015D800EF5F03C0E894F1F8E0E0E0931A03A0910C
:1015E8001A03A43109F025C1AA81E0E00E94FF276F
:1015F8000E2E0E947E21E02119F0EA81E150EA8353
:10160800233610F423E615C121E0E0E0E0930F0350
:10161800E0911103A0E0B0E00E94A822E09112033B
:10162800A1E0B0E00E94A822E0911303A2E0B0E09C
:101638000E94A822E0911503A3E0B0E00E94A8222E
:10164800EF89A4E0B0E00E94A822E88DA5E0B0E010
:101658000E94A822E98DA6E0B0E00E94A822E091AD
:101668001603A7E0B0E00E94A822E0911703A8E0C3
:10167800B0E00E94A822E0911803A9E0B0E00E941F
:10168800A822E0911B03AAE0B0E00E94A8220E94D1
:101698008F20A6E2B0E00E946522EB89A4E1B0E0C9
:1016A8000E94A822EC89A5E1B0E00E94A822ED8959
:1016B800A6E1B0E00E94A822EF85ABE0B0E00E946E
:1016C800A822E889ACE0B0E00E94A822E989ADE050
:1016D800B0E00E94A822ED81FE81AAE2B0E00E945B
:1016E8006522E0912803AEE0B0E00E94A822E091D4
:1016F8002A03AFE0B0E00E94A822E0912903A0E10C
:10170800B0E00E94A822E32FA1E1B0E00E94A82245
:10171800E985FA85ACE2B0E00E946522EB8DA2E192
:10172800B0E00E94A822EA8DA3E1B0E00E94A822BE
:101738000E946B220E94AE22A0E3B0E00E946522C4
:10174800E0915D03F0915E03A4E3B0E00E9465229E
:10175800E0E023FCE1E0A7E1B0E00E94A8220E94BB
:101768001120A2E3B0E00E946522E0910803A8E1FD
:10177800B0E00E94A822E0910A03A9E1B0E00E942B
:10178800A822E0910B03AAE1B0E00E94A822E09110
:101798000C03ABE1B0E00E94A822E0910D03ACE19C
:1017A800B0E00E94A822E0910E03ADE1B0E00E94F3
:1017B800A8220E945C1F0E94EE1F0E947822E091DE
:1017C8001F03AEE1B0E00E94A822E0912003AFE140
:1017D800B0E00E94A822E0912103A0E2B0E00E94BC
:1017E800A822E0912203A1E2B0E00E94A822E091A1
:1017F8002303A2E2B0E00E94A822E0912403A3E21E
:10180800B0E00E94A822E0912503A4E2B0E00E9483
:10181800A822E0912603A5E2B0E00E94A8220E9437
:10182800491FA8E3B0E00E9465220E94DA1FE1E0A8
:101838004E2E0E949722A0E0F1FCA1E00E949D227A
:10184800AA81E4E60E94FA270E94B32251F0689424
:10185800F1F8EA81EF5FEA83AA81A43611F4E0E0A7
:10186800EA83EAE0E91510F4E894F0F80E94782198
:101878000E9483210E22AA81E0E00E94F5270E949F
:10188800B32251F06894F0F8EA81E150EA83AA8122
:10189800AF3F11F4E3E6EA830E94D4200E94BA2203
:1018A800C1F00E94C022A9F4A0913103A43119F417
:1018B800E7E0E0933103E0E0E0933203E894F3F8E3
:1018C800A0913103A33028F0E0913103E150E09377
:1018D8003103AA2DEAE00E9404280E2E0E94BA22A3
:1018E800C1F00E94C022A9F4A0913103A43119F4D7
:1018F800E7E0E0933103E0E0E0933203E894F2F8A4
:10190800A0913103A33028F0E0913103E150E09336
:101918003103AA2D0E947D22AD2DEAE00E940928FC
:10192800E02131F0E0E0E0933203E4E1E0933103B9
:10193800EAE0ED1510F4E894F3F80E94D4200E9430
:10194800DA200E94EB27E02109F45BC26894F3F8DF
:10195800AA81A13049F4A0911103A13028F4E091A3
:101968001103EF5FE0931103AA81A23049F4A0911B
:101978001203A23328F4E0911203EB5FE093120301
:10198800AA81A33049F4A0911303A43628F4E09166
:101998001303EF5FE0931303AA81A43049F4A091E5
:1019A8001503A83228F4E0911503EF5FE0931503BF
:1019B800AA81A53031F4AF89A43618F4EF89EF5F16
:1019C800EF8BAA81A63031F4A88DA43618F4E88DDF
:1019D800EF5FE88FAA81A73031F4A98DA43618F4F7
:1019E800E98DEF5FE98FAA81A83049F4A091160329
:1019F800AF3F28F4E0911603EF5FE0931603AA8146
:101A0800AD3069F4A0913D03B0913E03A433E8E002
:101A1800BE0728F40E948F2031960E945720AA8181
:101A2800AE3031F4AB89A43618F4EB89EB5FEB8B5D
:101A3800AA81AF3031F4AC89A43618F4EC89EB5F95
:101A4800EC8BAA81A03131F4AD89A43618F4ED8964
:101A5800EB5FED8BAA81A13131F4AF85A83C18F476
:101A6800EF85EB5FEF87AA81A23131F4A889A83C02
:101A780018F4E889EB5FE88BAA81A33131F4A989CE
:101A8800A83C18F4E989EB5FE98BAA81A43169F4D1
:101A9800A0914D03B0914E03A835E2E0BE0728F4AB
:101AA8000E9411207E960E947120AA81A53159F4C6
:101AB800AD81BE81A33AE1E0BE0728F4ED81FE8145
:101AC8003196ED83FE83AA81A63149F4A0912803BB
:101AD800A13028F4E0912803EF5FE0932803AA815E
:101AE800A73149F4A0912A03A23328F4E0912A03EC
:101AF800EF5FE0932A03AA81A83149F4A091290352
:101B0800A13028F4E0912903EF5FE0932903AA812B
:101B1800A93119F43F3008F43F5FAA81AA3159F47A
:101B28000E94CB22AC3BE2E0BE0728F40E94AE2222
:101B380031960E946320AA81AB3191F40E94D02291
:101B4800A73EE3E0BE07E0E08E07E0E09E0740F432
:101B58000E94281FEF5FFF4F6F4F7F4F0E94682042
:101B6800AA81AC3161F4A0E023FCA1E0A13038F4F3
:101B7800E0E023FCE1E0EF5F0E94682923F8AA81F6
:101B8800AD3169F40E94E81EAE3DE3E0BE0738F4CB
:101B98000E94C91E3A96E0934503F0934603AA8132
:101BA800AE3169F40E94F21EA835E2E0BE0738F4AF
:101BB8000E94D51E3A96E0935103F0935203AA81EE
:101BC800AF3149F4A0910803AA3028F4E091080342
:101BD800EF5FE0930803AA81A03249F4A0910A03B9
:101BE800AB3028F4E0910A03EF5FE0930A03AA817F
:101BF800A13249F4A0910B03AB3028F4E0910B0318
:101C0800EF5FE0930B03AA81A23249F4A0910C0381
:101C1800AB3028F4E0910C03EF5FE0930C03AA814A
:101C2800A33249F4A0910D03AB3028F4E0910D03E1
:101C3800EF5FE0930D03AA81A43249F4A0910E034B
:101C4800AB3028F4E0910E03EF5FE0930E03AA8116
:101C5800A53249F4A0911F03A13028F4E0911F0395
:101C6800EF5FE0931F03AA81A63249F4A0912003F5
:101C7800A13028F4E0912003EF5FE0932003AA81CC
:101C8800A73249F4A0912103A13028F4E09121035F
:101C9800EF5FE0932103AA81A83249F4A0912203BF
:101CA800A13028F4E0912203EF5FE0932203AA8198
:101CB800A93249F4A0912303A13028F4E091230329
:101CC800EF5FE0932303AA81AA3249F4A091240389
:101CD800A33028F4E0912403EF5FE0932403AA8162
:101CE800AB3249F4A0912503A13028F4E0912503F3
:101CF800EF5FE0932503AA81AC3249F4A091260353
:101D0800A13028F4E0912603EF5FE0932603AA812F
:101D1800AD3291F40E94E01FAF39E6E8BE07E1E07A
:101D28008E07E0E09E0740F40E94C81FE65FFF4F61
:101D38006F4F7F4F0E94D11FAA81AE3259F40E9483
:101D4800D922A031E7E2BE0728F40E94491F3A963B
:101D58000E944E1FAA81AC3549F4A0910703AA3FFF
:101D680028F4E0910703E65FE0930703AA81AD3505
:101D780031F4AC8DA73018F4EC8DEF5FEC8FAA81AD
:101D8800AE3549F4A985BA851A9728F4E985FA8504
:101D98003196E987FA87AA81AF3531F4AB8DAA303D
:101DA80018F4EB8DEF5FEB8FAA81A03631F4AA8D82
:101DB800AA3018F4EA8DEF5FEA8FAA81A13649F4B8
:101DC800A0911B03AC3328F4E0911B03EF5FE09371
:101DD8001B03AA81A23649F4A0911803AA3F28F44C
:101DE800E0911803E65FE0931803AA81A33649F44B
:101DF800A0911703AA3F28F4E0911703E65FE09348
:101E08001703EAE0EA1510F4E894F2F8AA2DEAE0DC
:101E18000E9404280E2E0E948F220E94BA2209F4E2
:101E280051C26894F2F8AA81A13049F4A091110333
:101E3800A13028F0E0911103E150E0931103AA8149
:101E4800A23049F4A0911203AB3028F0E0911203BC
:101E5800E550E0931203AA81A33049F4A09113033B
:101E6800AD3328F0E0911303E150E0931303AA8106
:101E7800A43049F4A0911503A53128F0E091150389
:101E8800E150E0931503AA81A53031F4AF89A13060
:101E980018F0EF89E150EF8BAA81A63031F4A88DB4
:101EA800A13018F0E88DE150E88FAA81A73031F40D
:101EB800A98DA13018F0E98DE150E98FAA81A830E9
:101EC80049F4A0911603A13028F0E0911603E150DF
:101ED800E0931603AA81AD3069F4A0913D03B09157
:101EE8003E03AD36E7E0BE0728F00E948F20319709
:101EF8000E945720AA81AE3031F4AB89A63018F081
:101F0800EB89E550EB8BAA81AF3031F4AC89A63070
:101F180018F0EC89E550EC8BAA81A03131F4AD8939
:101F2800A63018F0ED89E550ED8BAA81A13131F486
:101F3800AF85A13018F0EF85E550EF87AA81A2316F
:101F480031F4A889A13018F0E889E550E88BAA8116
:101F5800A33131F4A989A13018F0E989E550E98B5A
:101F6800AA81A43161F4A0914D03B0914E030E945F
:101F7800542928F40E9411207E970E947120AA817A
:101F8800A53159F4AD81BE81A332E1E0BE0728F046
:101F9800ED81FE813197ED83FE83AA81A63149F454
:101FA800A0912803A13028F0E0912803E150E093A4
:101FB8002803AA81A73149F4A0912A03A23028F066
:101FC800E0912A03E150E0932A03AA81A83149F459
:101FD800A0912903A13028F0E0912903E150E09372
:101FE8002903AA81A93119F4323008F03150AA81A5
:101FF800AA3159F40E94CB22A935E2E0BE0728F0A5
:102008000E94AE2231970E946320AA81AB3191F4DD
:102018000E94D022AB30E0E0BE07E0E08E07E0E0AF
:102028009E0740F00E94281FE150F0406040704039
:102038000E946820AA81AC3179F4A0E023FCA1E0D9
:10204800A13050F0A0E023FCA1E0E1E00E941529B6
:10205800EA1B0E94682923F8AA81AD3161F40E9425
:10206800E81E0E94542938F40E94C91E3197E09353
:102078004503F0934603AA81AE3161F40E94F21E33
:102088000E94542938F40E94D51E3197E0935103D9
:10209800F0935203AA81AF3149F4A0910803A2300A
:1020A80028F0E0910803E150E0930803AA81A032E8
:1020B80049F4A0910A03A23028F0E0910A03E15004
:1020C800E0930A03AA81A13249F4A0910B03A1303D
:1020D80028F0E0910B03E150E0930B03AA81A232B0
:1020E80049F4A0910C03A13028F0E0910C03E150D1
:1020F800E0930C03AA81A33249F4A0910D03A13007
:1021080028F0E0910D03E150E0930D03AA81A43279
:1021180049F4A0910E03A13028F0E0910E03E1509C
:10212800E0930E03AA81A53249F4A0911F03A130C0
:1021380028F0E0911F03E150E0931F03AA81A63223
:1021480049F4A0912003A13028F0E0912003E15048
:10215800E0932003AA81A73249F4A0912103A1307A
:1021680028F0E0912103E150E0932103AA81A832ED
:1021780049F4A0912203A13028F0E0912203E15014
:10218800E0932203AA81A93249F4A0912303A13044
:1021980028F0E0912303E150E0932303AA81AA32B7
:1021A80049F4A0912403A13028F0E0912403E150E0
:1021B800E0932403AA81AB3249F4A0912503A1300E
:1021C80028F0E0912503E150E0932503AA81AC3281
:1021D80049F4A0912603A13028F0E0912603E150AC
:1021E800E0932603AA81AD3259F40E94DE2240F022
:1021F8000E94C81FEA50F040604070400E94D11F02
:10220800AA81AE3249F40E94D9221A9728F00E9476
:10221800491F3A970E944E1FAA81AC3539F4A09104
:102228000703A13018F0E0E0E0930703AA81AD3579
:1022380031F4AC8DA13018F0EC8DE150EC8FAA810F
:10224800AE3551F4A985BA850E94542928F4E98548
:10225800FA853197E987FA87AA81AF3531F4AB8DD2
:10226800A13018F0EB8DE150EB8FAA81A03631F444
:10227800AA8DA13018F0EA8DE150EA8FAA81A13623
:1022880049F4A0911B03A13028F0E0911B03E15011
:10229800E0931B03AA81A23649F4A0911803AB303E
:1022A80028F0E0911803EA50E0931803AA81A336B6
:1022B80049F4A0911703A13028F0E0911703EA50E0
:1022C800E093170323FC26C0E0912F03ABEBB3E0A8
:1022D800FF27662777270E9462260E940229A0917D
:1022E800BB03B091BC038091BD039091BE030E94D3
:1022F80058293CF40E94E7220E94F0220E94F7220B
:1023080009C0E0E0E093AB03E093AC03E093AD03D6
:10231800E093AE0323FE0BC0AD850E940023ABEB18
:10232800B3E00E945C200E94E7220E94F7220E94EC
:10233800E722ADE2B3E00E942926EC93F091530323
:10234800E0E0DF01E0913003F0E0EA0FFB1FABE8CB
:10235800B3E00E94CE1E0E940623A0E0B0E080E118
:1023680092E40E943A277F936F93FF93EF930E9422
:10237800CB220E940F23AF91BF918F919F910E9412
:102388000622E0938B03F0938C0360938D03709384
:102398008E030E941423E0E0F0E060E87FE30E94EF
:1023A800A5270E2E0E941423E0E0F0E068E472E412
:1023B8000E949F27E021E9F00E9406230E94F02254
:1023C800A7E7B3E00E942B260E9402290E94062359
:1023D800E0938F03F09390036093910370939203BB
:1023E8000E9414230E94EE1FAFE3B3E00E94001F77
:1023F80015C0E0E0E0937703E0937803E093790376
:10240800E0937A03E0938F03E0939003E0939103C2
:10241800E0939203E0933F03E0934003A091AF035E
:10242800B091B0038091B1039091B2030E94E91F6B
:102438000E94A527EF930E941D230E94A527AF9114
:10244800EA23B9F10E94161FE0E0F0E068EC72E4BC
:102458000E943A270E94D0220E9407290E94441F06
:102468000E941F23A0918703B0918803809189035C
:1024780090918A03E0E0F0E064E172E40E94EC26C7
:10248800DF01CB010E94891F0E943A27A0E0B0E03B
:1024980080E291E40E94EC260E941F23E0918703CA
:1024A800F09188036091890370918A03DE010E948C
:1024B8007D1F0E947821A0911903EDEF0E94042846
:1024C8000E220E947E21E02129F0E0911903EF5F9E
:1024D800E0931903A92D0E947D22A0911903EFEF23
:1024E8000E9404280E220E947E21E02129F0E8940F
:1024F800F0F8E0E0E0931903A0911903EEE10E94DF
:10250800EB270E2E0E947E21E02119F0E1E0E093F6
:102518001C03E0911B03E03019F4E0E0E0931C0396
:102528000E94F71F0E94E91F0E9436280E945D2220
:10253800A0911C03E0E00E940928E02119F0E1E0E5
:10254800E0931C03A0911C03AC3309F41FEFA09186
:102558000703A13028F0E0910703F0E00E94C520AE
:102568004420C9F4E02FF0E034960E94AA20AE0F70
:10257800BF1FE12F0E942823A4E00E94AA1EA02FBB
:102588000E943223A09135030E94AA1EA12F0E9407
:10259800AA1E0E943723E1E0E41509F057C044243D
:1025A800A09113030E944023E0931403F0E0BC962B
:1025B800DF01E0911003F0E0AE0FBF1FE0911103BF
:1025C800F0E0AE0FBF1FE0911203F0E0AE0FBF1FA7
:1025D800E0911503F0E0AE0FBF1FEF89F0E0AE0FFA
:1025E800BF1FE88DF0E0AE0FBF1FE98DF0E0AE0F22
:1025F800BF1FE09116030E942823ACE20E94AA1E86
:10260800A09110030E94AA1EA09111030E94AA1E65
:10261800A09112030E94AA1EA09114030E94AA1E50
:10262800A09115030E94AA1EAF890E94AA1EA88D18
:102638000E94AA1EA98D0E94AA1EA09116030E949C
:102648003223A0E00E9432230E943723233608F069
:1026580002C40E94A2222081A0E0F799A1E0EA2FFB
:10266800E295E07F0E2EA0E0F399A1E0EA2FEE0FAD
:10267800EE0F0E0EA0E0F499A1E0EA2FEE0FA02DC8
:10268800AE0FE0E0F599E1E0EA0FED8FEAE0EAABA2
:10269800EBABECABEDABEEABEFABE8AF0E94462398
:1026A800EAE0ECAFEDAFEEAFEFAFDE01A05CBF4FFD
:1026B800EC93E0912403E03021F40E944B23E00DD9
:1026C800EE8FA0912403A13081F4A0E022FCA1E0C8
:1026D800EA2FEE0FE75F0E2EA0E022FCA1E0EA2F22
:1026E800EE0FEE0FE00D0E946423A0912403A230A8
:1026F80099F40E944B230E0EA0E022FCA1E0EA2FE1
:102708000E947E230E0EA0E022FCA1E0EA2FE295B3
:10271800E07FEE0FE00DEE8FA0912403A33031F49B
:10272800E0E022FCE1E0E85F0E9464230E9483234A
:10273800AA34E1E0BE07E0E08E07E0E09E071CF463
:10274800E1E0E09302030E948323E9E4F1E060E022
:1027580070E00E948C23EEE5F1E060E070E00E94FA
:102768002E28E02119F0E3E0E09302030E9483237E
:10277800EDE5F1E060E070E00E948C23E8E6F1E02E
:1027880060E070E00E942E28E02119F0E7E0E09375
:1027980002030E948323E7E6F1E060E070E00E9414
:1027A8008C23ECE7F1E060E070E00E942E28E02145
:1027B80019F0EFE0E09302030E948323AC37E1E0D5
:1027C800BE07E0E08E07E0E09E071CF0EFE1E09333
:1027D80002030E94F71F0E9490232CF00E94982366
:1027E8000E949E23ECAB0E9498230E94CD28EDAB5B
:1027F800A0912D03AA3028F00E9400230E94A9234B
:10280800EAAB0E94AF23EBAB0E9483230E94B7235D
:102818000E949E23EEAB0E94BC230E949E23EFAB36
:102828000E94BC230E94CD28E8AF2130A1F5EF8D8E
:10283800E056EF8F0E94C2230E94CC23A436E0E02A
:10284800BE0720F00E94CC230E94D1230E94CC23F3
:102858000E940F230E94DC230E94E2230E94CC23C3
:102868000E94E823DB01EC93A0910103AA3010F049
:10287800E2E0E9AFA09101030E94ED23EAAFA09145
:1028880000030E9400230E94A923EBAFA09100033C
:102898000E94ED23ECAF223009F050C0EF8DE05CD0
:1028A800EF8F0E94E01FA03AE6E8BE07E1E08E073E
:1028B800E0E09E0748F00E94E01FE0EAF6E861E0E9
:1028C80070E00E94F323EBAF0E94E01F0E94FE23FA
:1028D80048F00E94E01FE0E1F7E260E070E00E944B
:1028E800F323ECAF0E94E01F0E94062438F00E94F8
:1028F800E01F0E946D210E94F323EDAF0E94E01FAC
:102908000E940E2438F00E94E01F0E94B7230E9404
:10291800F323EEAF0E94DE2228F00E9416240E94C4
:10292800F323EFAFFE01F1963F96FF93EF930E94DA
:1029380016240E94C928AF91BF91EC93233009F067
:1029480077C0E7E7EAAFE4E7EBAFA0918603AA23F5
:1029580092F4E0918303F091840360918503709170
:1029680086030E94B927E0938303F093840360935E
:102978008503709386030E941D230E94441F7723BA
:1029880012F4E0E4EFAF0E941D230E94441F0E944E
:102998001C2410F4E0E4EEAF0E941D230E94441FA3
:1029A8000E94252410F4E0E4EDAF0E941D230E944C
:1029B800441F0E942E2410F4E0E4ECAF0E94372458
:1029C8000E94FE234CF00E943724E0E1F7E260E029
:1029D80070E00E949E23ECAF0E9437240E940624D8
:1029E8003CF00E9437240E946D210E949E23EDAF87
:1029F8000E9437240E940E242CF00E9437240E9443
:102A08004024EEAF0E9437240E9490232CF00E94AD
:102A180042240E949E23EFAFFE01F1963F96FF935A
:102A2800EF930E9442240E94CD28AF91BF91EC936E
:102A3800243009F04BC00E944824A0916C03AA23BB
:102A480012F40E9450240E945B24772312F4E0E4DD
:102A5800EFAF0E945B240E941C2410F4E0E4EEAF68
:102A68000E945B240E94252410F4E0E4EDAF0E944C
:102A78005B240E942E2410F4E0E4ECAF0E94612451
:102A8800A031E7E2BE071CF00E946624ECAF0E946A
:102A98006124A83EE3E0BE071CF00E946C24EDAF61
:102AA8000E946124A436E0E0BE071CF00E94722454
:102AB800EEAF0E9461241A972CF00E9478240E949D
:102AC8007C24EFAF0E947F240E9484242530C9F41F
:102AD8000E944824E0E5ECAFA0912C03A43618F03E
:102AE8000E948924EEAFA0912C030E9400230E942B
:102AF800A9230E94E223A0912C030E94ED23DB016D
:102B0800EC93263069F5EF8DE058EF8FE0E0EAAFFF
:102B1800E5E0EBAFE8E7ECAFA881B981A83EE3E0D8
:102B2800BE072CF0E8EEF3E00E947C24EDAFA8810C
:102B3800B981A436E0E0BE072CF0E4E6F0E00E949C
:102B48007C24EEAFA881B981EAE0F0E00E947C2401
:102B58000E94E223A881B981EAE0F0E00E9484247F
:102B6800273009F043C0113010F1ECE0EAAFA12F93
:102B78000E944023E436A0E0FA073CF0A12FB0E021
:102B8800E8ECF0E00E947C24EBAFA12F0E944023E8
:102B98003A973CF0A12FB0E0E4E1F0E00E947C24F9
:102BA800ECAFA12F0E9440230E94A9231EC0EBE096
:102BB800EAAF0E948F24E436A0E0FA0738F0AB8130
:102BC800BC81E8ECF0E00E949424EBAF0E948F24D3
:102BD8003A9738F0AB81BC81E4E1F0E00E9494249C
:102BE800ECAF0E948F240E94DC23EDAF283009F05F
:102BF80074C00E94C223A0916703B0916803A135F5
:102C0800EBEFBE0734F4E1E5FBEFE0936703F093E5
:102C18006803A0916703B0916803A03BE4E0BE0796
:102C280034F0EFEAF4E0E0936703F0936803A091CF
:102C38006803AA234AF4E0E4EDAFE0916703F0915A
:102C480068030E94B52704C0E0916703F091680308
:102C5800E0936903F0936A03A0916903B0916A0352
:102C6800ECE3F0E00E948928E0934703F0934803DF
:102C78000E949724ECE30E946628A0916903B09112
:102C88006A03AE1BBF0BA0934903B0934A0324FE0B
:102C98001BC00E9497241A9710F0E2E0E9AF0E9447
:102CA80097240E94E823EAAFA0914903B0914A0310
:102CB8000E940F230E94DC23EBAFA0914903B0913F
:102CC8004A030E94E823ECAFE3E7EEAFE8E3EFAF97
:102CD800E4E5DE01A05CBF4FEC93293009F04BC05E
:102CE8000E949C24A0916C03AA2312F40E945024F1
:102CF8000E945B24772312F4E0E4EFAF0E945B2488
:102D08000E941C2410F4E0E4EEAF0E945B240E94B1
:102D1800252410F4E0E4EDAF0E945B240E942E24E9
:102D280010F4E0E4ECAF0E946124A031E7E2BE07B2
:102D38001CF00E946624ECAF0E946124A83EE3E0E8
:102D4800BE071CF00E946C24EDAF0E946124A436DB
:102D5800E0E0BE071CF00E947224EEAF0E946124DE
:102D68001A972CF00E9478240E947C24EFAF0E94CE
:102D78007F240E9484242A30C9F40E949C24E0E520
:102D8800ECAFA0912C03A43618F00E948924EEAF72
:102D9800A0912C030E9400230E94A9230E94E223F1
:102DA800A0912C030E94ED23DB01EC932B3061F5FD
:102DB800EF8DE054EF8FE9E3EBAFE8E3ECAF0E946F
:102DC800D922A83EE3E0BE0738F00E94D922E8EEF7
:102DD800F3E00E949424EDAF0E94D922A436E0E0EB
:102DE800BE0720F00E94D9220E94D1230E94D92236
:102DF8000E940F230E94DC230E94E2230E94D92212
:102E08000E94E823DB01EC93AC85A130E8F0EF8D5C
:102E1800EF77EF8FE0912E03E170EE0FAE8DEA238E
:102E2800EE8F0E944623E9E7ECAFE0E5EDAFEEAFA9
:102E3800AC850E9400230E94A9230E94E223AC854E
:102E48000E94ED23DB01EC93F29B05C0EE8DEB7F36
:102E5800EE8FEF5FEE8F233609F069C451E05031F1
:102E680030F40E94A624EAE0EC935F5FF8CFAA81D1
:102E7800EBE50E94AD24EAE50E94EB27E02911F07A
:102E8800EEE2EA83AA81AF3211F4ECE5EA83EA8143
:102E9800E03029F4E0911003F0E0EF83F887AA818D
:102EA800A13029F4E0911103F0E0EF83F887AA81BB
:102EB800A23029F4E0911203F0E0EF83F887AA81A9
:102EC800A33029F4E0911303F0E0EF83F887AA8197
:102ED800A43029F4E0911503F0E0EF83F887AA8184
:102EE800A53021F4EF89F0E0EF83F887AA81A630B6
:102EF80021F4E88DF0E0EF83F887AA81A73021F468
:102F0800E98DF0E0EF83F887AA81A83029F4E091F1
:102F18001603F0E0EF83F887AA81A93019F4E0E0FE
:102F2800EF83E887AA81AA3019F4E0E0EF83E88705
:102F3800AA81AB3019F4E0E0EF83E887AA81AC30CE
:102F480021F4E4E2F0E0EF83F887AA81AD3021F4C0
:102F58000E948F20EF83F887AA81AE3021F4EB8995
:102F6800F0E0EF83F887AA81AF3021F4EC89F0E034
:102F7800EF83F887AA81A03121F4ED89F0E0EF838F
:102F8800F887AA81A13121F4EF85F0E0EF83F88773
:102F9800AA81A23121F4E889F0E0EF83F887AA81B9
:102FA800A33121F4E989F0E0EF83F887AA81A431FD
:102FB80021F40E941120EF83F887AA81A53121F41A
:102FC800ED81FE81EF83F887AA81A63129F4E0918B
:102FD8002803F0E0EF83F887AA81A73129F4E0916C
:102FE8002A03F0E0EF83F887AA81A83129F4E09159
:102FF8002903F0E0EF83F887AA81A93121F4E32FB0
:10300800F0E0EF83F887AA81AA3121F40E94AE226A
:10301800EF83F887AA81AB3131F4E0915D03F09139
:103028005E03EF83F887AA81AC3131F4E0E023FC3A
:10303800E1E0F0E0EF83F887AA81AD3121F40E9446
:10304800C91EEF83F887AA81AE3121F40E94D51EEC
:10305800EF83F887AA81AF3129F4E0910803F0E003
:10306800EF83F887AA81A03229F4E0910A03F0E0FF
:10307800EF83F887AA81A13229F4E0910B03F0E0ED
:10308800EF83F887AA81A23229F4E0910C03F0E0DB
:10309800EF83F887AA81A33229F4E0910D03F0E0C9
:1030A800EF83F887AA81A43229F4E0910E03F0E0B7
:1030B800EF83F887AA81A53229F4E0911F03F0E095
:1030C800EF83F887AA81A63229F4E0912003F0E083
:1030D800EF83F887AA81A73229F4E0912103F0E071
:1030E800EF83F887AA81A83229F4E0912203F0E05F
:1030F800EF83F887AA81A93229F4E0912303F0E04D
:10310800EF83F887AA81AA3229F4E0912403F0E03A
:10311800EF83F887AA81AB3229F4E0912503F0E028
:10312800EF83F887AA81AC3229F4E0912603F0E016
:10313800EF83F887AA81AD3231F4E0915903F09119
:103148005A03EF83F887AA81AE3221F40E94491FFF
:10315800EF83F887AA81AC3529F4E0910703F0E002
:10316800EF83F887AA81AD3521F4EC8DF0E0EF8389
:10317800F887AA81AE3521F4E985FA85EF83F887C7
:10318800AA81AF3521F4EB8DF0E0EF83F887AA81AF
:10319800A03621F4EA8DF0E0EF83F887AA81A13602
:1031A80029F4E0911B03F0E0EF83F887AA81A236A7
:1031B80029F4E0911803F0E0EF83F887AA81A33699
:1031C80029F4E0911703F0E0EF83F887AA81E0E0A3
:1031D8000E94AD24E3E00E94B224E1E10E94B224FF
:1031E800E2E10E94B224E3E10E94B224E5E10E94F8
:1031F800B224EBE10E94B224EDE10E94B224EEE297
:103208000E94EB27E02911F0F69A01C0F698A0E099
:10321800F699A1E0EA2FE795E0E0E795EF8FE0E087
:10322800EE8FED8FE09302030E94B7240E947C2466
:10323800ECAB0E94B7240E94BB28EDABAF81B885E8
:10324800A031E7E2BE0728F0E0E1F7E20E9494240B
:10325800ECAFAF81B885A83EE3E0BE0728F0E8EE02
:10326800F3E00E949424EDAFAF81B885A436E0E086
:10327800BE0710F00E94D123AF81B8851A9728F0B5
:103288000E94BE240E94DC23EFAFFE01F1963F9618
:10329800BF01AF81B8850E94E823DB01EC93EA8186
:1032A800E03061F4EDE6EEABE9E7EFABE8E7E8AF75
:1032B800EDE6EBAFE4E5ECAFE0E5EDAFAA81E1E1E7
:1032C8000E94AD24E2E10E94B224E3E10E94B2240C
:1032D800E5E10E94B224EDE10E94B224EEE20E94F0
:1032E800EB27E02929F00E94BE240E94DC23EFAFDF
:1032F800E7EAE0937A000E949B20E7E2E0937A00F5
:10330800AA810E94CA20AA81EEE00E94B224E1E1CB
:103318000E94EB27E02911F0E1E06E2EAA810E94BD
:10332800CF20AA81EFE00E94B224E2E10E94EB27BD
:10333800E02911F0E2E06E2EAA81E7E00E94AD24B8
:10334800E0E10E94B2240E94C12411F0E3E06E2E55
:103358000E94AA20D39708F457C00E94E4200E9434
:10336800E920E62D0E94F02020F0E8ECF0E00E9431
:10337800C520E62D0E9400210E94C624AC91A130F0
:1033880008F441C00E94CD240E9420210E94632994
:103398004CF40E94C6240E94D6240E94AB270E94A7
:1033A800E12423C00E94EA240E944221EF930E9454
:1033B800EA240E944B21AF91EA2379F00E94C624A7
:1033C8000E94D6240E94B027A0937303B09374037D
:1033D800809375039093760308C00E94EA240E94A4
:1033E80054211CF00E94EC240EC0A0917303B091EC
:1033F800740380917503909176030E946D210E9459
:10340800B3280E94C52004C00E9472210E94EC24A7
:10341800AA81AD3051F40E94F4240E9440240E94F5
:10342800FD240E940425E0E2ED8FAA81A53151F424
:103438000E94F4240E9440240E94FD240E94042536
:10344800E0E6ED8FAA810E94CA20AA81EEE00E94E0
:10345800B224E1E10E94EB27E029A9F00E940E25A1
:10346800E4E00E94122518F00E941825EEAB0E9495
:10347800AA201A9728F00E941C250E94DC23EFAB93
:103488000E941E25E8AFAA810E94CF20AA81EFE002
:103498000E94B224E2E10E94EB27E029A9F00E94F1
:1034A8000E25E2E00E94122518F00E941825EEABC6
:1034B8000E94AA201A9728F00E941C250E94DC234B
:1034C800EFAB0E941E25E8AFAA81E7E00E94AD2479
:1034D800E0E10E94B2240E94C124A9F00E940E25B6
:1034E800E1E00E94122518F00E941825EEAB0E9418
:1034F800AA201A9728F00E941C250E94DC23EFAB13
:103508000E941E25E8AFAA81A43199F40E942025C3
:10351800E4E6F0E00E949424EEAB0E9420250E948D
:103528000F230E94DC23EFAB0E9420250E94E82392
:10353800E8AFAA81A63121F40E942525EBE0EDAF82
:10354800AA81A73121F40E942525E0E4EDAFAA81E4
:10355800A83121F40E942525ECE0EDAFAA81A9311C
:1035680061F4A0912D030E9400230E94A923EEABD1
:103578000E94AF23EFABE7E7E8AFAA81AA3199F43D
:103588000E942C25E4E6F0E00E949424EEAB0E9411
:103598002C250E940F230E94DC23EFAB0E942C25D0
:1035A8000E94E823E8AFAA81AB3159F4ECE7EAAF0F
:1035B800E7E7EBAFE8E7ECAF0E94BE240E94DC230C
:1035C800EFAFAA81EDE10E94AD24EEE10E94EB2766
:1035D800E029D9F0E3E7EAAFE8E3EBAFAA81AD3140
:1035E80011F4EEE501C0E8E7ECAF0E9431251A9727
:1035F80038F00E9431250E940F230E94DC23EFAB94
:103608000E9431250E94E823E8AFAA810E94CA20BF
:10361800AA81E6E00E94B224E7E00E94EB27E029B5
:1036280011F0E3E7EAAFAA81EEE00E94AD24EFE0F3
:103638000E94B224E0E10E94EB27E02931F0EDE698
:10364800EAAFE9E7EBAFE4E5ECAFAA81E1E10E947C
:10365800AD24E2E10E94B2240E94C12411F0E8E7FF
:10366800EBAFAA81EFE10E94FF270E2EE5E20E9450
:10367800FA27E02139F0EDE6EEABE8E5EFABEA81B9
:10368800EF51E8AFAA81AD3219F4EF8DE05CEF8F0E
:10369800AA81AE3221F4E9E3EBAFE8E3ECAFAA810B
:1036A800AD3559F5E7E7EDAFEEE5EEAFE9E3EFAF9E
:1036B800FE01F1963F96AC8DA083E7EAE0937A008D
:1036C8000E94A5207E2EE7E2E0937A00E3E6E71564
:1036D80038F4A72DB0E0E4E6F0E00E947C24EEABDD
:1036E800E9E0E71530F4A72D0E9400230E94A923E2
:1036F800EFABA72D0E94ED23E8AFAA81AE3521F4E8
:10370800EEE5EAAFE1E0EBAFAA81AF3521F4EEE5F3
:10371800EAAFE2E0EBAFAA81A03621F4EEE5EAAF2A
:10372800E3E0EBAFAA81A23611F4E0E1ED8F51E0BE
:10373800503108F077C00E94A624EC91E03021F4C3
:103748000E94A624EFE3EC930E94A624AC91A63035
:1037580021F40E94A624EDE7EC930E94A624AC91E4
:10376800A13021F40E94A624E6E0EC930E94A6244E
:10377800AC91A23021F40E94A624EBE5EC930E94C0
:10378800A624AC91A33021F40E94A624EFE4EC9384
:103798000E94A624AC91A43021F40E94A624E6E657
:1037A800EC930E94A624AC91A53021F40E94A62493
:1037B800EDE6EC930E94A624AC91A73021F40E9478
:1037C800A624E7E0EC930E94A624AC91A83021F44B
:1037D8000E94A624EFE7EC930E94A624AC91A9309E
:1037E80021F40E94A624EFE6EC930E94A624AC9153
:1037F800AA3021F40E94A624E0E0EC930E94A624BB
:10380800AC91AB3021F40E94A624E1E0EC930E9435
:10381800A624AC91AC3021F40E94A624E8E0EC93F5
:103828005F5F86CFE0910203E695E6950E94362514
:10383800EEA90E943C25EEA90E944425EEA90E940B
:103848004F25EEA90E945625EEA90E945D25EEA9F6
:103858000E946425EEA90E946B25E9A3E09102036A
:10386800E695E695E6950E943625EFA90E943C2547
:10387800EFA90E944425EFA90E944F25E8AD0E94B8
:103888005625E8AD0E945D25E8AD0E946425E8ADA7
:103898000E946B25EAA3E0910203E6950E94362573
:1038A800E8AD0E943C25E8AD0E944425E8AD0E94A1
:1038B8004F25EFA90E945625EFA90E945D25EFA983
:1038C8000E946425EFA90E946B25EBA3E9AD0E9435
:1038D8003625EAAD0E943C25EAAD0E944425EAADB2
:1038E8000E944F25EF8D0E945625EF8D0E945D2581
:1038F800EF8D0E946425E0910203E170EA2BECA3AE
:10390800EEAD0E943625EEAD0E947125EEAD0E9407
:103918007725EEAD0E9480250E948A25EEAD0E9493
:103928008E25EEAD0E949725EEADE295E170EA2B6B
:10393800EDA3EDAD0E943625EDAD0E947125EDADEC
:103948000E947725EDAD0E948025E2950E945625BC
:10395800EFAD0E948E25EFAD0E949725EFADE29561
:10396800E170EA2BEEA3EF8D0E94A025EDAD0E9439
:103978003C25EDAD0E944425EDAD0E944F25ECADF0
:103988000E945625ECAD0E945D25ECAD0E94642591
:10399800ECAD0E946B25EFA3EFAD0E943625EFAD8D
:1039A8000E947125EFAD0E947725EFAD0E9480251A
:1039B8000E94A4250E945625ECAD0E948E25ECADF0
:1039C8000E949725ECADE295E170EA2BE8A7EBADF4
:1039D8000E943625EBAD0E947125EBAD0E9477253C
:1039E800EBAD0E948025EE1FE0E0EE1F0E945625F9
:1039F8000E94A9250E948E250E94A9250E9497252C
:103A08000E94A925E295E170EA2BE9A7EE8DE295DF
:103A18000E943625EBAD0E943C25EBAD0E94442563
:103A2800EBAD0E944F25EAAD0E945625EAAD0E94F3
:103A38005D25EAAD0E946425EAAD0E946B25EAA7E0
:103A48000E94A9250E9436250E94A9250E94712559
:103A58000E94A9250E9477250E94A925E695E6954A
:103A6800E6950E94AE25EAA9EE1FE0E0EE1F0E944F
:103A78005625EAA9E2950E94B425EAA90E9497254D
:103A8800EAA9E295EF70E695E170EA2BEBA7EAA9BF
:103A9800E695E695E6950E943625EAA9E695E69527
:103AA8000E94BA25EAA90E94BF25EAA90E94AE256C
:103AB800EE8D0E948A25EE8D0E94C725EE8D0E940C
:103AC800CA25EE8DE695E170EA2BECA7EE8D0E94F3
:103AD800A025EBA9E2950E94BA25EBA90E944425EE
:103AE800EBA90E94CF25EBA90E948A25EBA90E9489
:103AF800C725EBA9E6950E94CA25EBA9E170EA2B38
:103B0800EDA7EE8D0E94A4250E943625ED8D0E941A
:103B1800BA25ED8D0E94BF25ED8DE695E6950E94AC
:103B2800AE25E0910203E2950E945625EE8DEE1F28
:103B3800E0E0EE1F0E94B425ED8DE695E695E6954A
:103B48000E94CA25ED8DE295E170EA2BEEA7ED8D76
:103B58000E94A025ECA9E2950E94BA25ECA90E9432
:103B68004425ECA90E94CF25EDA90E948A25EDA93C
:103B78000E94C725EDA9E6950E94CA25EDA9E17026
:103B8800EA2BEFA7ED8D0E94A4250E943625EDA90A
:103B9800E2950E94BA25EDA90E944425EDA90E944C
:103BA800CF25ECA90E948A25ECA90E94C725ECA97B
:103BB800E6950E94CA25ECA9E170EA2BE8AB33FE32
:103BC8000DC051E0513150F4E52FF0E0DE01909640
:103BD800AE0FBF1FEFEFEC935F5FF4CF0E94D325CA
:103BE8005D3078F40E94D925A2E5B8E00E94C92783
:103BF800E17011F45D9801C05D9A0E94E0255F5F55
:103C0800EFCF0E94E8255D3078F40E94D925A0E323
:103C1800B8E00E94C927E17011F45D9801C05D9A6F
:103C28000E94E0255F5FEFCF0E94E8255D3078F4C1
:103C38000E94D925A2E0B8E00E94C927E17011F4DA
:103C48005D9801C05D9A0E94E0255F5FEFCF0E94FA
:103C5800E8255D3078F40E94D925A6E0B8E00E94F6
:103C6800C927E17011F45D9801C05D9A0E94E025B2
:103C78005F5FEFCF0E94E8255A3098F45E9885E29E
:103C88008A95F1F7E9E0E51BA0E4B1E00E94C927B5
:103C9800E17011F45D9801C05D9A0E94E0255F5FB4
:103CA800EBCF41E04131E8F451E05930C0F45E987F
:103CB80085E28A95F1F7E42FF0E0DE019096AE0FE9
:103CC800BF1FAC91E8E0E51B0E94C127E17011F429
:103CD8005D9801C05D9A0E94E0255F5FE6CF4F5F67
:103CE800E1CF5D9A85E28A95F1F7289A8DEC9AE002
:103CF8000197F1F70E947821A82DEAE00E94042894
:103D08000E2AAA2DEAE00E9404280E2AAD2DEAE028
:103D18000E940428E02929F0E0E0E0934F03E093B3
:103D28005003AB2DE4E60E9409280E2EA0E0F0997E
:103D3800A1E00E949C2139F0A4E6B0E00E94F2259F
:103D4800F09AE89433F80C946605FFCFAA93E091B3
:103D5800C000E072E1F3E881E093C600219608957F
:103D6800A0913903B0913A030895A0918F03B091BF
:103D7800900380919103909192030895E0E0F0E020
:103D880061EE75E40E943A270895E0914503F091A9
:103D980046030895662777270E9462260E94022913
:103DA8000895E0915103F09152030895A09197036B
:103DB800B09198038091990390919A030895E0E057
:103DC800F0E060E271E40895A0914503B0914603E4
:103DD8000895E0E0F0E00E9420280895A0915103A2
:103DE800B09152030895E091BF03F091C003609130
:103DF800C1037091C20308950E942926ED93FC9394
:103E08000895A091AB03B091AC038091AD0390915C
:103E1800AE03E0E0F0E06AE774E40E94EC26DF011C
:103E2800CB01ACCFA091A703B091A8038091A903BF
:103E38009091AA030895A091CB03B091CC038091EF
:103E4800CD039091CE030895E0915D03F0915E0358
:103E580060915F03709160030895A4E6B0E080E08C
:103E680090E00E944628DF01CB01E091A703F09182
:103E7800A8036091A9037091AA030E9407290895D5
:103E88000E940C290E9495260895E0915703F0910D
:103E980058030895E0935703F09358030895E09169
:103EA8007B03F0917C0360917D0370917E030895FC
:103EB800A091C703B091C8038091C9039091CA0328
:103EC8000895E093C703F093C8036093C903709300
:103ED800CA0308950E944628DF01CB01E091C70379
:103EE800F091C8036091C9037091CA030E94072921
:103EF800C7CF0E942B26ED93FC930895E0E0F0E0F5
:103F080061EE75E40E94EC260895E091AF03F0910C
:103F1800B0036091B1037091B2030895E091B303C7
:103F2800F091B4036091B5037091B6030895A09120
:103F38009303B0919403809195039091960308950B
:103F4800E0939303F093940360939503709396031F
:103F58000895A0919B03B0919C0380919D0390913B
:103F68009E030895E0919303F09194036091950363
:103F7800709196030895A091A303B091A403809132
:103F8800A5039091A6030895E0915903F0915A036F
:103F980060915B0370915C030895E0935903F0937B
:103FA8005A0360935B0370935C030895EDDFAAE303
:103FB800B0E00E942D290895A0915903B0915A03A9
:103FC80080915B0390915C030895E0E0F0E060E08D
:103FD80070E00895F4DE0E94EC260895E0E00E9467
:103FE80009280E2E0895A0917703B0917803809147
:103FF800790390917A0308950E22A0911C03ECE3B3
:104008000E9404280895A0914F03B0915003089589
:10401800A0914D03B0914E03DCCEE0914D03F09199
:104028004E030895E7EAE0937A00A4E00E945E0355
:10403800EF2FF0E09E2EE7E2E0937A00E7EAE093C4
:104048007A000895A3E00E945E03EF2FF0E08E2E21
:10405800E7E2E0937A00E7EAE0937A000895A1E0C6
:104068000E945E03EF2FF0E0AE2EE7E2E0937A00C5
:104078000895E0E0F0E00E9435290895EBE0E09330
:10408800D403E8EBE093D5030895E8ECF0E0E0937F
:104098006303F09364030895E0EDF7E0E0936503AC
:1040A800F09366030895E0933D03F0933E0308956B
:1040B8000E94E1270E9462260E9402290895E09347
:1040C8004303F09344030895E0935D03F0935E0384
:1040D80060935F03709360030895E0934D03F0933A
:1040E8004E030895E7EAE0937A00A0E00E945E0399
:1040F800EF2FF0E008950E945E030E94D6270E94E9
:10410800D2270895E0937B03F0937C0360937D03AB
:1041180070937E030895E0913D03F0913E03089566
:10412800E7E2E0937A00E7EAE0937A000895A7E0EF
:104138000E945E03EF2FF0E0E0933503F09336031F
:1041480008950E945E03EF2FF0E00895A0913503D3
:10415800B09136030895FADFEAEFF0E00895F6DF4C
:10416800EEE1F0E00E941A2808950E2EA52DE1E058
:104178000E9409280E22AC85E5E00E940428E0216F
:104188000895E0933503F09336030895E5E00E941F
:10419800EB270E2E0895E6E00E94EB270E2E0895D9
:1041A800AD2DEAE00E9404280E2E0895A0E0F3FC4D
:1041B800A1E0E0E00E94EB270E22A22FE3E608959B
:1041C800E0913503F09136030895F297ADE7B0E03A
:1041D8000E943E280F010895F0E0DE015296AE0FCE
:1041E800BF1FEC91F0E0D0010E947628CADFAEDF55
:1041F800A93CE0E0BE070895F0E0DE015696AE0F58
:10420800BF1FEC91F0E0A2DF0E943E28DF01E4E648
:10421800F0E00E947628B5CFE02FF0E0DE011E9690
:10422800AE0FBF1F0895A0916F03B09170038091E6
:104238007103909172030895E8EEF3E060E070E096
:104248000E94B328DF01CB01BBDF662777270895DB
:10425800EC91F0E00E94E127A8E0BCE481E090E066
:104268000E94B328E0CFE0936F03F093700360934C
:104278007103709372030895D6DFDECF0E94B027D2
:10428800E5E0F0E060E070E00E94362808950E94C2
:10429800B027E4E1F0E060E070E00E942E28089585
:1042A8000E94B027A431E0E0BE07E0E08E07E0E01E
:1042B8009E070895E0917703F09178036091790360
:1042C80070917A03A0E5B4E180E090E00E94712843
:1042D800CACFE8EEF3E060E070E00895E0E0E09334
:1042E8003503E09336030895A92DEAE00E940428D7
:1042F8000E2E0895A22FE3E60E9404280895A0E058
:10430800F0FCA1E0E0E00E94EB270895A0E022FC89
:10431800A1E0E0E00E94EB27E0210895A0912B03A3
:104328005DCEE0912A035FDEFF2766277727089591
:10433800E0E00E94EB27E0210895ED81FE81A09145
:104348007B03B0917C0380917D0390917E03662767
:1043580077270E942E280E2EEAE0F0E060E070E059
:104368000E9436280895E0936303F0936403089548
:1043780096DDAD81BE81882799270E94B0270895D0
:10438800A630E0E0BE07E0E08E07E0E09E07089573
:10439800A0916303B09164030895E0916303F091E1
:1043A80064030895ED81FE81A0917B03B0917C03A5
:1043B80080917D0390917E03662777270895E32FE8
:1043C800A091BB03B091BC038091BD039091BE0343
:1043D800FF27662777270E9462260895B7DEEAE05E
:1043E8000E9466280895E32FF0E0A091BB03B091E6
:1043F800BC038091BD039091BE030E94E1270E94F7
:1044080062263ECD662777270E9462260E94EC2608
:104418000895A0916503B091660308950E94E62768
:104428000E9409292DCDA32FBB27E091BB03F09152
:10443800BC036091BD037091BE03F0CFE0916503AA
:10444800F09166030895EAE0F0E00E94892899CE89
:10445800E0911203C8DDFF27662777270895E093C8
:104468006D03F0936E030895E0911203F0E0BBDD55
:104478000E94E1270E94B02708950E946C28A0910D
:104488006D03B0916E030895E0916D03F0916E0392
:104498000895A0911203BB27E0917703F091780368
:1044A8006091790370917A030E94E6270E94B027F1
:1044B80008950E2EA0911C03ECE30E9404280E22FE
:1044C80008950E943529A1E0B0E00C94F225E0910E
:1044D800A703F091A8036091A9037091AA03AEE223
:1044E800B0E00E942B26EDCFA6E3B0E00E942B2679
:1044F800E8CFEAE00E9409280E2E0895AA2DEAE0E6
:104508000E9404280E2EA0E027FCA1E0E0E00E9413
:10451800EB270E220895A0E0F2FCA1E0E0E00E9463
:10452800EB270E220895A82DEAE00E9404280E2EFB
:104538000895E0E00E94EB270E220895E0910F0312
:10454800F0E0E65FFC4F08950E943D29A1E0B0E04D
:104558000C94F225E0914303F091440308950E2250
:10456800A22FE3E60E94EB27E0210895A22FE3E6BD
:104578000E94EB27E0210895E0913203EF5FE0937A
:104588003203E0913103A0913203EA170895A09114
:104598004303B09144030895A0915D03B0915E0375
:1045A80080915F03909160030895A0915703B091A3
:1045B8005803089501DDAA30E0E0BE07E0E08E0769
:1045C800E0E09E070895E091BB03F091BC03609181
:1045D800BD037091BE030895A0E0B0E080E09FE3C2
:1045E8000E949C260895E093AB03F093AC0360937C
:1045F800AD037093AE030895B0E0EAE0F0E00E94E6
:1046080089280895E0918B03F0918C0360918D03C4
:1046180070918E030895EAE0F0E00E9476280895EC
:10462800A0918B03B0918C0380918D0390918E03A0
:1046380008950ADC12CCE0938703F0938803609313
:10464800890370938A030895F0E0EA0FFB1FE09353
:104658004103F0934203AEE30C94AA1E0E94AA1EE3
:10466800A0E00C94AA1EE0914203AE2F0E94AA1E5D
:10467800A09141030C94AA1EB0E0E2E0F0E00E9491
:1046880089280895EAE0E9AFEAAFEBAF0895E9E0D9
:10469800EF8FE0912E03E170EE0FE058AE2FE0911E
:1046A8002E03E695E695E170EE0FEE0FEA0F0E2E5B
:1046B800A0E0F199A1E0EA2FEE0FEE0FEE0F0895BA
:1046C800EF8FE0912E03E170EE0FE058AE2FE091EE
:1046D8002E03E695E695E170EE0FEE0FEA0F0E2E2B
:1046E800A0E0F199A1E0EA2FEE0FEE0FEE0FE00D3A
:1046F800EE8F0895E295E07FEE0FEE0F0895A091FA
:104708007F03B09180038091810390918203089583
:104718000E9436280E2EF3CFAA30E0E0BE07E0E074
:104728008E07E0E09E0708955EDCEAE0F0E060E0D6
:1047380070E008950E94B328DF01CB01EAE0F0E0C1
:1047480060E070E00E94CD280895DF01EAE0F0E023
:104758000E94BB280895A0912D03BB27EAE0F0E052
:104768000E94BB280895E4E6F0E060E070E0089558
:10477800C6DFEAE0F0E060E070E00895A0E020FC29
:10478800A1E0EA2FE295E07FAE8DEA0FEE8F089563
:10479800A0913B03B0913C030895E4E6F0E00E9449
:1047A8007628DF01EAE0F0E00E94B828EEAF08952D
:1047B800DF01EAE0F0E00E94B8280895EFAFFE01BB
:1047C800F1963F96BF010895EAE0F0E00E94B8280C
:1047D8000895BB27EAE0F0E00E94BB2808950E94F4
:1047E8008E28DF01CB01EAE0F0E060E070E00E9493
:1047F800C9280895A031E7E2BE07E0E08E07E0E0AF
:104808009E070895A83EE3E0BE07E0E08E07E0E0DB
:104818009E070895A436E0E0BE07E0E08E07E0E0DA
:104828009E070895C9DBEAE0F0E060E070E00895D3
:10483800DF01CB01E0E0F0E060E171EC0E947F274E
:104848000895DF01CB01E0E0F0E066EC72EC0E9435
:104858007F270895DF01CB01E0E0F0EC69E774EC15
:104868000E947F270895A0918303B09184038091CB
:10487800850390918603089576DF5CCFF4DFEAE044
:10488800F0E060E070E00895EF8DE058EF8FEEE320
:10489800EAAFE4E7EBAF0895E0916B03F0916C03A6
:1048A8000E94B527E0936B03F0936C030895CCDA6C
:1048B800A4E6B0E080E090E00DCBA0916B03B0914E
:1048C8006C030895FADFE0E1F7E20E9489283DCF02
:1048D800F4DFE8EEF3E00E94892837CFEEDFE4E664
:1048E800F0E00E94892831CFE8DFEAE0F0E008959F
:1048F8000E9489282ACFFE01F1963F96BF01F4CF86
:104908000E94BB28DB01EC930895A0912C03B0E032
:10491800E4E6F0E0EDCFEB81FC81F695E7950895AC
:104928000E94762845CFA0914703B0914803089587
:10493800EF8DE058EF8FE2E0E9AFEEE3EAAFE4E7AE
:10494800EBAF0895E52FF0E0DE01D196AE0FBF1F63
:1049580008950E94EB270E2EAA8108950E94EB2746
:104968000E2AAA810895AA81B0E0A7FDBFEFEAE068
:10497800F0E00895AF81B8854ECEE3E10E94EB27C1
:10498800E0290895E62DF0E0DE011E96AE0FBF1F68
:104998000895A0917303B091740380917503909169
:1049A80076030895EC91F0E00E94E127A8E0BCE4CA
:1049B80081E090E00E94B328ECCFE0937303F0937A
:1049C800740360937503709376030895E2DF34CC23
:1049D800E985FA8508DB662777270E947128EDCFDD
:1049E800A0917B03B0917C0380917D0390917E031D
:1049F8000895EEABF5DFEAE0F0E060E070E09ACE13
:104A0800EFABEEDFEAE0F0E060E070E00E94CD2876
:104A1800E8AF0895D5DBF695E795B3CBED8F96DB38
:104A2800A436E0E0BE07089591DBE4E6F0E078CF35
:104A38008DDBF1CD8BDBC8CEA0915503B091560329
:104A48000895E9E3EAAFE0E5EBAFEEE3ECAF0895F4
:104A5800A0913F03B09140030895A0914B03B091FA
:104A68004C030895E170E795E0E0E795AE2F0895CF
:104A7800E295EF70E695E1703DDEEA2BAE2F0895E2
:104A8800E295EF70E695E695E170E295E07FEE0F2E
:104A9800EA2BAE2F0895E295E170E295E07FEA2BCC
:104AA800AE2F0895E170EE0FEE0FEE0FEA2BAE2F4A
:104AB8000895E695E170EE0FEE0FEA2BAE2F0895FC
:104AC800E695E695E170EE0FEA2BAE2F0895E69590
:104AD800E695E695E170EA2B0895E695E1700ADE21
:104AE800EA2BAE2F0895E695E695E170E295E07F12
:104AF800EE0FEA2BAE2F0895E695E695E695E17060
:104B0800E295E07FEA2BAE2FEF8D0895E695E695C6
:104B1800E695C8CFE295EF70E695E170EE0FEE0FDF
:104B2800EA2BAE2F0895E295EF70E695E695E170D1
:104B3800EE0FEA2BAE2F0895E295EF70E69592CF2F
:104B4800E295EF70E695E6950895FE01E05CFF4F6B
:104B5800E0810895E170E295E07FEA2BAE2F089599
:104B6800E170EE0FEE0FEA2BAE2F0895E170C2DD73
:104B7800EA2BAE2F0895E695E170E295E07FEE0FFF
:104B8800EA2BAE2F0895E695E695EACFE170EE0F91
:104B9800EA2BAE2F0895E295EF70E695DBCF2898C3
:104BA80085E28A95F1F751E008955E9885E28A9545
:104BB800F1F7ECE0E51B089585E28A95F1F75E9A36
:104BC80085E28A95F1F708955D9A85E28A95F1F76D
:104BD800289A84E191E00197F1F7E1CF109639F036
:104BE8008DEC9AE00197F1F7A8951197C9F7089508
:104BF800552342F4503811F4E0FF04C03196691F80
:104C0800791F6BF050E8572711F45F93CFC05F3FCF
:104C180031F0660F000C57956795752F08955F93CF
:104C280000200AF0CFC0C8C050E8192E1522880FFE
:104C3800991F9527550F879550E8072E0522660F6F
:104C4800771F7527550F67950895689401C0E894F4
:104C58005F93F2DF703818F07F3F08F4A7C056E181
:104C6800571BAAF4519558300EF4593030F0EFEF35
:104C7800FFEF6FEF7FE777F91AC077275523B9F071
:104C8800EE0FFF1F661F771F5A95D1F710C07727C1
:104C9800583028F0EF2FF62F672F5850F9CF5523AB
:104CA80031F076956795F795E7955A95D1F70020F5
:104CB8000AF45BD15F910895689401C0E894309735
:104CC80060407040B1F0002426F0772312F400947D
:104CD8004CD1172E7EE1112032F07A95EE0FFF1F8E
:104CE800661F111CF9CFEF2FF62F612D5F938ADF16
:104CF8005F9108954F93AF01FD01DA01AB01BC014B
:104D0800CA01402D012C142E4F910895EA0FFB1F64
:104D1800681F0895E095F0956095EF5FFF4F6F4F1E
:104D280008955F9381DF903871F150E8152604C02B
:104D38005F937ADF903839F1703821F1572F591B7A
:104D48002BF112F4D7DFFACF583118F0AA27BB2776
:104D58008827583028F0AB2FB82F88275850F9CF1C
:104D6800552329F08695B795A7955A95D9F7502DCB
:104D7800512572F0CBDF38F46795F795E795739571
:104D880013F420C0B7DF3EDF5F910895D8F7FBCF5B
:104D9800EA1BFB0B680B51F010F40094BBDF662391
:104DA80092F3EE0FFF1F661F7A95CBF7EE27FF27CA
:104DB800662777275F910895EFEFFFEF6FE77FEFA3
:104DC8005F910895EFEFFFEF6FE77FE75F91089539
:104DD8005F932ADF703851F3903841F30124089427
:104DE800791F23F41CF300203AF3ECCF0F921F93A2
:104DF8002F933F934F93112722279927689FA0014C
:104E08008F9F302D410D591F6B9F300D411D591F2C
:104E18008E9F27D0BF9F25D06A9F23D0BE9F1DD0CD
:104E2800AF9F1BD0AE9F110D291F391F491F591F56
:104E3800E32FF42F652F522F4F913F912F911F9100
:104E48000F9066232AF0550FEE1FFF1F661F02C042
:104E580073954BF2CDDE5F910895100D211D391F1A
:104E680002C0200D311D491F591F08955F93DCDED4
:104E7800703821F411200AF49FCFA4CF903809F498
:104E880095CF01240894970B1BF4D4F30020F3CF9B
:104E9800792F1F932F933F934F9311241127222784
:104EA80033274427552790E2AE17BF0786074107E7
:104EB80030F0AE1BBF0B860B410B089401C08894E1
:104EC800551F221F331F111CAA1FBB1F881F441FF9
:104ED8009A9551F7F901612D4F913F912F911F91AB
:104EE800662332F0550FEE1FFF1F661F7A9543F2B7
:104EF8007FDE5F91089599239AF0772342F0971700
:104F080048F029F4AE17BF07860720F031F09894CF
:104F18008894089598940894089518948894089506
:104F28007723C2F7971798F3A9F7EA17FB076807DB
:104F380088F399F3ECCFDFDFE1E009F008F0EE2722
:104F48000895D9DFE1E009F008F4EE270895EA0FA3
:104F5800FB1F681F791F0895AE1BBF0B860B970BAD
:104F68000895F195E195F0400895F0956095709554
:104F7800E195FF4F6F4F7F4F0895EE230E2EEA2FD6
:104F880019F0E6950A94E9F70895EE230E2EFD012F
:104F980021F0F695E7950A94E1F70895F695E795D7
:104FA800F695E795F695E795F695E7950895FE2F1A
:104FB800FF0FFF0B6F2F7F2F08956F2F660F660B64
:104FC800762F08958B2F880F880B982F0895EA174E
:104FD800E1E009F0EE270895EA17E1E009F4EE2789
:104FE8000895AE17E1E00CF4EE270895AE17E1E05E
:104FF8000CF0EE270895EA17E1E00CF0EE2708958B
:10500800AE17E1E008F0EE270895EA17E1E008F0AE
:10501800EE270895EA17FB07E1E009F0EE27089567
:10502800AE17BF07E1E008F4EE270895AE17BF07F3
:10503800E1E008F0EE270895EA17FB07E1E008F041
:10504800EE270895EA17FB0768077907E1E009F0FA
:10505800EE270895AE17BF0786079707E1E00CF023
:10506800EE270895EA17FB0768077907E1E00CF0D7
:10507800EE270895FA9FF02DEB9FF00DEA9FE02DA3
:10508800F10D08957A9F702D6B9F700DF89F700D2C
:10509800E99F700D6A9F602D710DFB9F600D711D5A
:1050A800E89F600D711D8827FA9FF02D610D781F0C
:1050B800EB9FF00D611D781FEA9FE02DF10D681F31
:1050C800781F08956E2F6A9FF0016B9FF00D089569
:1050D80074D0D0DF0EF445DF08957DD0D3DF0EF411
:1050E80044DF08950024112490E1AA0FBB1F001C7F
:1050F800111C0E1A1F0A18F40E0E1F1E01C0A16003
:105108009A9599F7FD01D001089557D0EBDF0EF479
:1051180028DF08953F934F935F9300241124442779
:10512800552730E2AA0FBB1F881F991F001C111CAE
:10513800441F551F0E1A1F0A460B570B28F40E0E54
:105148001F1E461F571F01C0A1603A9559F7FD0160
:10515800BC01D001CA015F914F913F9108953BD0A6
:10516800D9DF0EF402DF0895BDDFFD010895E8944C
:10517800B7FF04C0A095B09511966894F7FDF1DECD
:10518800B1DFFD010EF4EDDE0895C4DFFD01BC01C1
:105198000895E89497FF09C0A095B09580959095DB
:1051A800AF5FBF4F8F4F9F4F689477FDDEDEB2DF52
:1051B800FD01BC010EF4D9DE0895E894F7FF02C0A2
:1051C800D0DE6894B7FF06C0A095B095119600F898
:1051D800039400FA0895E89477FF02C0C6DE689445
:1051E80097FF0BC00024A095B095809590951196D7
:1051F800801D901D00F8039400FA0895ED93FD9327
:105208006D937C930895689401C0E89401D057DDAC
:10521800182E862F612D192E972F712D1B2EBF2F1B
:10522800F12D1A2EAE2FE12D0895129602D0BF014E
:105238001297119602D0FE2F1197F999FECFFF937E
:10524800FFB7F894A1BDB2BDF89AE0B5FFBFFF91D2
:10525800089507D012960F01FB0103D0F0011297B1
:10526800089507D01196EF93EF2F03D0EF91119780
:105278000895F99B02C0A895FCCF9FB7F894A1BDEB
:10528800B2BDF89A80B5E81719F0E0BDFA9AF99A14
:105298009FBF089500240E160F06060607060895F8
:1052A80000240A160B06089500240A160B060806A1
:1052B80009060895EA17FB07680779070895AE17E6
:1052C800BF07860797070895E894EE2309F06894C6
:1052D8000895AC0FBD1F05900D928A95E1F70895CA
:00000001FF
